:0200000480007A
:10000000971F0000938F0F00171100001301810349
:1000100083A10F0023203100171C0000130CDCFE0D
:100020009712000093824202832CFCFF23A09201CE
:1000300097130000938373FD171400001304040149
:1000400083AF13002320F401171500001305457C2E
:10005000971500009385C5FF0326058023A0C500E2
:10006000970600009386167B17170000130787FE7C
:1000700083A7F67F2320F70017180000130808FA5B
:1000800097180000938848FD0329C8FF83290800BA
:10009000032A480023A0280123A2380123A44801F1
:1000A000971A0000938A0AF8171B0000130B8BFBAA
:1000B00003A00A0023200B00971A0000938ACAF6B7
:1000C000171B0000130B4BFA83AB0A0003AC0B00A9
:1000D000930C0C0023209B01971C0000938C4CF583
:1000E000171D0000130D8DF883AC0C0023209D011B
:1000F000971D0000938D1DF4171E0000130E4EF780
:1001000083ADFDFF2320BE0117150000130585F305
:1001100097150000938505F6370610F01306C6F212
:100120006306B5028326C5002320D60083268500FA
:100130002320D600832645002320D60083260500F1
:100140002320D600130505016FF09FFD370510F041
:10015000130505F223200500000000000000000048
:04016000000000009B
:1010000022F2F111F44433F366F6F555F88877F7D8
:10101000AA0A09990CCCBB0BEE0E0DDDF000FF0FF8
:101020007856341228100080F0DEBC9A10325476C4
:1010300098BADCFE00000000000000000000000084
:10104000FFFFFFFFFFFFFFFFFFFFFFFFFFFFFFFFB0
:10105000FFFFFFFFFFFFFFFFFFFFFFFFFFFFFFFFA0
:10106000FFFFFFFFFFFFFFFFFFFFFFFFFFFFFFFF90
:040000058000000077
:00000001FF
